:020000000328D3
:1000060083128F018C018316850186018312850177
:1000160086010C08043A031D112830280C08C1007B
:100026000130C000410803191C28C00D4010FF3ED6
:1000360016280508C004400885008C0A0430CB0049
:100046000C30CC003330CD00CD0B2728CC0B272825
:10005600CB0B2728000000000C280F08083A031DC8
:10006600482883128F018C01860185010430CB005C
:100076000C30CC003330CD00CD0B3F28CC0B3F28C5
:10008600CB0B3F28000000000C280F08C1000130F0
:10009600C000410803195328C00D4010FF3E4D28EB
:1000A60083120608C004400886008F0A0430CB007D
:1000B6000C30CC003330CD00CD0B5F28CC0B5F2845
:0C00C600CB0B5F280000000030286828E9
:02400E00F23F7F
:00000001FF
